:020000000150AD
:02000300012DCD
:02000B00012EC4
:020013000143A7
:02001B0001439F
:02002300014397
:10002B00014332C0E0758AE8758C03758810E5369C
:09003B00600314F536D0E0323206
:1000500075A8007581607580FF7590FF75A0FF75AC
:10006000B0FFC2B3C2B5C282C280C2817514F3753B
:1000700015FF751603D1C5120C7675A800D2B31101
:100080009920020530B30AD202D282D281D2808076
:1000900003120DEF120CC5017F30B20122C20275AE
:1000A00014F4D1CAE51420E02D20E12D20E22D200A
:1000B000E32C20E42BD282D280D2817514D0751526
:1000C00080D1C07514D1751500D1C07514D87515BF
:1000D00000D1C011E22202089A02086401FE21DB6D
:1000E0004134C2017531E075360075330075090081
:1000F000750E00752201752300C21DD21E227514D3
:1001000042D1CA751482D1CAE51430E50520E23027
:10011000800122751402F13F75300A7514F0D1E0A8
:10012000E5156016B40113E5317531E0B4320B8585
:1001300016587514F2F13FD162227514F2F13F2284
:10014000751403F13F7514F1F13F7514F2F13F7529
:100150001402F13F7514F1F13F75300A7514F0D1B6
:10016000E07514F2F13FE515B40869AA16AB17ACB7
:1001700018AF19AD1AAE1C8E37EB54F07056EA5416
:100180002003C0E0EB540FF531D0E0453123F531C9
:1001900090019473417641C2817561008175613E21
:1001A000615E61B061E361E461ED61EE61EF817513
:1001B00081758175817561F0813B81508175817593
:1001C00081758175817581658166816F81758175A4
:1001D00081758175D17ED189C19422751443D1CAAC
:1001E000E53154E064E0700122E531C2E0541F9033
:1001F00001F373817F81C9C10981FAC109A12BA1D2
:1002000046A19CA19DA1C3A1D8A1F3C102C109C16E
:1002100009C109C109C103C104C105C109C109C19D
:1002200009C109C109C106C107C108C109C109C184
:1002300009C10922751444D1CAE5367038E54E70FB
:10024000347514F075150075160885561775180065
:1002500085501985511A85521B85531C85541D855F
:10026000551E75300A120714E550600122E55660EC
:100270000122754E0122EA5403603F14600C1460A1
:10028000107531E0D17ED189C19474204531F531AA
:1002900022ED6018B4010280E87514841206CA7554
:1002A0005900E51430E30C7559018007755900D1E8
:1002B0009FD1AA74404531F5312274004531F531A2
:1002C0002222EA5403600F14601914601F7531E094
:1002D000D17ED189C194ECB401F3C21E74004531C2
:1002E000F5312241CD74204531F53122ECB400DDE9
:1002F000EDB4010774404531F53122D1B580F522C6
:10030000EA5403600F14601914601F7531E0D17E48
:10031000D189C194ECB401F3D21E74004531F5319A
:1003200022610B74204531F53122ECB400DDEDB4CF
:10033000010774404531F53122D19480F5227531A1
:10034000E08C33D1627514F4D1CAE51430E3F6754C
:1003500014D1E5334480F515D1C0750B0022EF149C
:10036000700774004531F53122147007742045314F
:10037000F5312214700674404531F531147007745C
:10038000604531F5312214700774804531F5312212
:10039000EFB4210774A04531F53122B4220774C0AF
:1003A0004531F53122B423047531E0227531E02264
:1003B000EC14700774004531F53122147007742075
:1003C0004531F5312214700674404531F531147011
:1003D0000774604531F5312214700774804531F59A
:1003E00031222222EC6003D21D22C21D22222222AF
:1003F0008519327531E0E53214600514602BC17E39
:100400007514F07515007516088556177518008552
:10041000501985511A85521B85531C85541D8555CD
:100420001E75300A754D00E1207514F075150075C4
:100430001601751700753003E120227531E075143F
:10044000F0751500751601853617753003E1202209
:100450007531E07514F0751500751601855717751F
:100460003003E12022228519367531E0D1622285E0
:100470001957D162227531E0D17ED189C19422E52C
:100480003120E044D2E0F53154E0C490049B75146F
:10049000F07515007516027518007381A181B2817F
:1004A000BD7531E07402201E025401F51775300449
:1004B000E1207531E0751700753004E1207531E0F9
:1004C000855917753004E12022E53120E02BD2E078
:1004D000F53154E0C49004D97381DF81E581EBD11B
:1004E000627531E022D1627531E0227531E0C217C8
:1004F000D162D1AAD19FD1B52222E53120E02BD201
:10050000E0F53154E0C490050A73A110A116A11CB6
:10051000D1627531E022D1627531E0227531E0D2CD
:1005200017D162D17ED189D1942222E53120E00712
:10053000D2E0F531D162227531E07514D1E5334452
:1005400080F515D1C022E53120E007D2E0F5317504
:10055000350054E0C490055973A167A16FA177A13C
:100560007CA184A18CA194900E1F753412C11090AF
:100570000E31753422C1107531E0C17E900E3A758E
:100580003409C110900E4C753407C110900E43759C
:100590003409C110900E5375343FC11022E531204B
:1005A000E020D2E0F5317514F0751500751601756F
:1005B00017007530037531E0201D02E12075170129
:1005C000E12022E53120E00FD2E0F5317531E0E5A0
:1005D000334480F533D16222E53120E015D2E0F5D5
:1005E000317514F075150075160175170075300317
:1005F000E12022E53120E009D2E0F5317531E0D18A
:10060000622222222222222222D17ED189C1942258
:10061000751483D1CAE51420E5477514F0751500EB
:10062000753000781779080530E535930535F608FB
:10063000E535B537057531E0C157B5340B54077052
:1006400002C1577531E0C157C39534400875160093
:10065000753003E120D9D07816A63005300530F189
:100660002022751403F13F7514F0751500751600FE
:10067000751700753003F12A7514FAF13F227514CD
:1006800043751501753001E12A7514427515017520
:100690003001E12A751444751501753001E12A75A0
:1006A0001443751500753001E12A75144275150063
:1006B000753001E12A751444751500753001E12A81
:1006C000753001E12A753002E12A753001C1F7E584
:1006D00014C0E0751400F13FD1CAD0E0F5148017C2
:1006E000E514C0E0E530C0E0751402F13FD1CAD096
:1006F000E0F530D0E0F514751336751201F15C7534
:100700001335853012F14822D201751401F13F757D
:1007100014F08016D201751404F13F7514F0800AAC
:10072000D201751403F13F7514F0F13F7513348550
:100730003012F15E3001077514FAF13FC2012275E3
:100740001336751201F15C22851211F17320000934
:100750007814F18BF608D511F9F1DD2278148512A1
:1007600011F17320000AE6F1B608200003D511F656
:10077000F1DD22C20030B11030B00DC2B0F1E8C2DC
:10078000B1F1E8E513F1B622D20022751008F1D7D5
:10079000F1E8A2B033C2B1F1E8D510F2C0E0E51142
:1007A000B40104D2B08002C2B0F1D7D0E0F1E8C207
:1007B000B1D2B0F1E8227510083392B0F1D7F1E868
:1007C000C2B1F1E8D510F2D2B0F1D7F1E830B00201
:1007D000D200C2B1F1E822D2B130B1FD22C2B0F1F3
:1007E000D7F1E8D2B0F1E82222E6C39408500CE633
:1007F000F92402F530750B00020802F50B79087533
:10080000300A75140112073F7514F075150089162A
:100810007817E493F608A3D9F985830C85820D1225
:1008200008612275300A0206F77530020206F77574
:1008300014417515011206C02275140112073F7587
:1008400014F075150075160075170012084F227503
:1008500030030207087530040207087530060207E6
:10086000080207087514411206CA7514011206CA57
:10087000E51454017023E50AB40510750A007514D7
:10088000D0E5094480F5151206C022780BE6600910
:10089000850C83850D821207E9227514401206CA61
:1008A0007514801206CAE5145404700122751401EF
:1008B00012073F7514F112073F75140012073F75B8
:1008C00014F112073F7514F01208237514F2120781
:1008D0003FE515B40802800122AA16AB17AC18AD8B
:1008E0001AAE1CEA54606003020A64EB601F1460D5
:1008F0001F1414601E1414603414601A1414604F12
:1009000014606514601714601012082F2202098801
:100910000209CB0209FD020A2F120839227514F0D0
:1009200075150075160175170012084F2278188684
:10093000091208397514F41206CAE51430E1F57588
:1009400014D0E5094480F5151206C0750B00227518
:1009500014F0751500751601751700200D041208A6
:100960004F2275170102095EEC6012B4019BD20D93
:100970007514D87515011206C012083922C20D75FA
:1009800014D87515000209767514F07515007516E2
:1009900002751700751800EA5403600914600C14FE
:1009A000600D020909E5215403F51712085522EDDF
:1009B00060F964806008ED6481600B020909300A07
:1009C000EA75170121AB300CE221C1EA600914601D
:1009D00003146009020909C20912083922ED60F9FD
:1009E00064806008ED64816010020909C20B75140F
:1009F000017515001206C021D9C20C21D9EA60097F
:100A0000146003146009020909D20912083922EDA1
:100A100060F964806008ED64816010020909D20BFE
:100A20007514417515011206C0410BD20C410BEC37
:100A300070D4E519B40114900F2A781C08E67007E9
:100A400018E6C39412401976124160B402B8900FB0
:100A50003C781C08E6700718E6C394194002761922
:100A60001207E922EB603314600F141460081414A9
:100A7000146009020909020BD2020AFDE519642972
:100A80007005900F5E418A900F55781CE6C394095B
:100A90004004760941961207E922ED601214601FA6
:100AA00014602B1460281460251460220209097553
:100AB00014E0120829E51503035402FEFF41DC751A
:100AC00014F77515001206C0AE22AF2341DCED14F9
:100AD0001444E0F514120829AE14AF157514F0751E
:100AE0001500751604EE541FF517EEC4035403F5F4
:100AF00018EF541FF519751A0012085B22300DAC5F
:100B0000ED605E147002616B14F954FC709EE94450
:100B1000E0F9EC14601C14601DC39406601CC394BF
:100B200008602114602214602314602414602502DC
:100B300009097E0061567E01615675220075230009
:100B40007E0361567E0461567E0561567E066156BF
:100B50007E0761567E0289148E151206C01208396E
:100B600022EC20E002612F79E06150EC14604F1418
:100B70006019C394066027C39408605214603B1444
:100B8000601814604914602C020909C212D21A7547
:100B900014F77515021206C061CEC21A61CE751423
:100BA000D17515001206C07514F77515021206C02E
:100BB00079E0613AC21C12083922C21961CE3011A3
:100BC0000DD219C2117514D17515001206C0120884
:100BD0003922300D21ED601E14603914F954FC7077
:100BE00015E944E8F9EC1460101460111414601154
:100BF00014141414600F0209097E0081127E018111
:100C0000127E028112D215D2107E0389148E151223
:100C100006C06156EC14603D14600D1414601F147E
:100C20001414146007020909D21281397514F7757A
:100C300015021206C079E881051208392222301502
:100C4000F87514F77515021206C0D21C750E00C295
:100C50001AC212815D3015E12011DED219D2117550
:100C600014D1E50E4480F5151206C07514D875151B
:100C7000031206C08139754E007524007557017541
:100C80008AE8758C0375890075881075A882C28200
:100C9000C280C281755000755100755200755300B5
:100CA000755400755500755600755800754D0075E2
:100CB0004600754700754800754900754A00754B38
:100CC00000754C0022B12DE5A0F46040AB24ACA02F
:100CD000791030240575240080020524B12DE5A08B
:100CE000FA7E01ECF45E600CEAF45E6007ECF45E00
:100CF0004AF4700CEEC3336003FE80E7D9D480065B
:100D00008B24B156A10C8B24B12DB1752024030581
:100D100024227524008546508547518548528549CF
:100D200053854A54854B55854C5691AC22D2B5D249
:100D300082D280D281E524202413B16CD2B4202346
:100D400006F5907580FF227590FFF580227590FF63
:100D50007580FFC2B422754601754701754801755B
:100D60004901754A01754B01754D0622E52454076A
:100D7000900E929322E5A0753908C3334002B184E6
:100D8000D539F8221539C0E0900E9AE524232323A3
:100D900054F84539936038F504900E0E7D08ED93B4
:100DA000B5040BED240893424C754E00A1CFDDEE47
:100DB0007406B54D04B1568016754E00E9C0E0ECDE
:100DC000C0E07446254DF9D0E0F7D0E0F9054D308C
:100DD000B318301E15E8C0E0EAC0E07514F67515CA
:100DE000001206C0D0E0FAD0E0F8D0E0053922E5E4
:100DF00058F4139282139281139280C2B52230313B
:100E0000323334353637383941424344454600E1C0
:100E1000E5E0E4E2E6E3E702200110044008801286
:100E2000010001000000087104020400010000003C
:100E30000109022200010100A005090400000103CC
:100E4000010100092100010001223F000705810383
:100E500008001205010906A101050719E029E71597
:100E6000002501750195088102950175088101959C
:100E70000575010508190129059102950175039170
:100E80000195067508150025650507190029658176
:100E900000C0FEFDFBF7EFDFBF7F4448463E3C420B
:100EA000403A1823240D100E361C1221260A053351
:100EB00038151320270919342C082F1F2D07066118
:100EC0005E1A564F314E4B555B625751314D4A5465
:100ED0005A635250654C4953595800E300000000D2
:100EE000000087948800E2E68B00E43900E000000F
:100EF00097008995E50096008AE128352A041D5F50
:100F00005C2B301E2E161B605D144347453D294166
:100F10003F3B0C22250B110F37170000000000008B
:100F2000E7000000000000000000120100010901BC
:100F300000087104010940000000000109021900C5
:100F4000010100A0050904000001090100000705D6
:100F500081030100FF0900050400300A020209298B
:070F6000050400300A020243
:00000001FF
